:10000000F89411240FEF0DBF00E10EBFA0E0B1E0A6
:10001000C3E2D1E0CA1BDB0B2196E2E5F1E02197B8
:1000200019F005900D92FBCFA3E2B1E0C3E2D1E05D
:10003000CA1BDB0B2196219711F01D92FCCF02D039
:100040000C9402F0CF92DF92EF92FF920F931F93E6
:10005000CF93DF9308E310E00F2EF3E3EF2EFF249E
:10006000F02D0F2EF2E3CF2EDD24F02D8FEF87BB86
:1000700014BA83E081BB0E94790080E091E00E9485
:100080009A00C1E0D0E0F801C0838D2F992787FD49
:100090009A958370F601808320E030E080E090E064
:1000A0000196F5E780339F07DCF32F5F3F4F253044
:1000B0003105A4F3F7018081992787FD909583701E
:1000C00090708130910549F4F2E0C030DF07D9F239
:1000D000CC0FDD1F8FE191E009C00297A1F6C1307E
:1000E000D10589F2D595C79581E291E00E949A00E9
:1000F000CACF109290008FE089B982E08BB988E175
:100100008AB986E0809395008F9A97988E98969AF0
:1001100008955F9904C097985F9BFECF979A8CB122
:10012000992787FD909508958699FECF5D9BFCCF1A
:100130008CB90895CF93DF93EC018881882331F047
:1001400089910E94940088818823D1F7DF91CF9113
:02015000089510
:100152007075736820627574746F6E20636F6E744D
:10016200726F6C6C6564206368617365720A002B40
:03017200002D005D
:00000001FF
